:100000000000012F0000000000000134000070001B
:10001000000001D0000001F400000338000002DC01
:1000200000007518000000000000769C0000049895
:10003000000004D80002625A000001000000000025
:1000400000000064000000C8000000010000000083
:10005000000000000000000000000000000000019F
:1000600000005B8D000000000000000000000000A8
:10007000000000000000013C00001E840000001091
:10008000000000000000000100000000000000006F
:10009000000000000000000000000001000000005F
:1000A000000000000000001A000000000000000036
:1000B0000000000000000000000000000000000040
:1000C0000000000000000000000000000000000030
:1000D000000000280040006D0010003000210001E9
:1000E000000300040005001E0000000000098968EC
:1000F0000089000000000000000000000000000077
:1001000000000000000000000000000000000000EF
:1001100000000000000000000000000000000000DF
:1001200000000000000000000000000000000000CF
:1001300000000000000000000000000000000000BF
:10035000000000000000000000000000000100009C
:100360000000000000000B4541B514BD421543AC30
:100370000B870BA80BC90BEA0C0B0C2C0C4D33A0F4
:1003800033FF0C6E0C8F0FE2106C10990B6611137B
:100390004FE911341006115C00000000000000005D
:1003A000000000000000000000000000000000004D
:1003B000000000000000000000000000000000003D
:1003C000000000000000000000000000000000002D
:1003D000000000000000000000000000000000001D
:1003E0000000000000000000000000000000040009
:1003F0000000000000008E6FFCBD089CCE001018AD
:10040000CE00002008A60018A7000818088C0010CD
:1004100025F3CC0017270BCE5E506F000883000138
:1004200026F8BD08A8BD5D7C20FB04FC0512DE0695
:100430003C9F064FF6045338DF0639DE063C9F0624
:100440004FF6045438DF0639DE063C9F064FF604AB
:10045000530505C3014E8FEC00C30001ED0038DFEA
:100460000639DE063C349F06BD3842DE06E701BD94
:10047000361BDE064FE6013138DF0639DE063C3436
:100480009F06DE06E701BD37C8CE045018DE061809
:10049000E6013A6D002637F70454C65C18A6013D04
:1004A000C3033CFD045A8DBA5D27234FF60454F76D
:1004B000045305050505C30498CE00103C3736CC1F
:1004C00004D8BD5C638D81CC000138382003CC009A
:1004D000FF3138DF0639DE063C9F068D85CC0001F2
:1004E00038DF0639DE063C9F06F60453C1012305BA
:1004F000CC000220045C8D844F38DF0639DE063CD8
:100500009F06F604532605CC000220055ABD057C43
:100510004F38DF0639DE063C9F06C602CE04526D18
:100520000027076F00CC000120085A095D2AF0CC93
:10053000000238DF0639DE063C3C9F06C60218CEB4
:100540000452DE061AEF01DE06EE016D00261EF1F2
:10055000045326098DA7C10127034F2021C6011886
:10056000DE0618EE0118E700CC000120115ADE0665
:100570001AEE0118091AEF015D26CCCC00023838BA
:10058000DF0639DE063C9F06DE083CDE0A3C7F00C3
:100590000B7D045726107D04562713F60338C5013A
:1005A000260CC602200FCC00FF20584F20557D049A
:1005B000592704C601D70BF60455D10B2302D70BDC
:1005C0007F0009CE04505FE7007C000908D609C10E
:1005D0000223F35FD709D10B240FBD06365D2BC66E
:1005E0007C0009D609D10B25F1F60453F1045824F7
:1005F0000FBD05E4C10126B3F60453F1045825F1FB
:10060000CC000138DF0A38DF0838DF0639DE063C67
:100610009F06DE083CDE0A3CDE0C3CDE0E3C18DFAA
:100620000418CEE66CCE00004F18DF0218DE041866
:10063000CE001ABD5CF44F5F8F840CC4008FDD0EBA
:10064000DF0C18DF0418DE0218EC02DD0A18EC00DB
:10065000DD08DC0ADE088F84F3C4FF8FDF08DC0EC0
:10066000DE0C9A0ADA0B8F9A08DA098F18ED02CDA0
:10067000EF0018DE0438DF0E38DF0C38DF0A38DF11
:100680000838DF0639DE063C3C9F06DE06ED01C673
:1006900003BD070D18CE0118183CDE06EE013CCC58
:1006A0000338BD5C6318CE0040183CDE06EE073C04
:1006B000CC0498BD5C637F0454CC033CFD045ABD5C
:1006C00005D618DE0618E60ABD070D7F0453CE00D6
:1006D000103C18CE0498183CCC04D8BD5C63BD0611
:1006E0008330C60C3A35CC00013838DF0639DE06D7
:1006F0003C9F06C1022305CC00FF2007F70455BD2F
:1007000006834F38DF0639DE063C9F06F604555C4B
:100710008DDC4F38DF0639DE063C9F06BD4272BDD8
:1007200006834F38DF0639DE063C9F068F8FC101F6
:100730008F2305CC00FF200DC602DF00D001F70497
:1007400058BD06834F38DF0639DE063C349F067FEE
:1007500001837F01827F01817F01805FF70454F76D
:100760000453CE01183C18CE70B8183CCC0338BDE9
:100770005C63F6045418DE0618E701C65C18A6018F
:100780003DC3033CFD045ACE005C3C3736CC02DC52
:10079000BD5C63383838383138DF0639DE063C9FB7
:1007A000060F4F5F38DF0639DE063C308FC3FFF29D
:1007B0008F359F06DE083CDE0A3CDE0C3CDE0E3C3C
:1007C000DE066F046F036F026F016F06CC5E6A84F2
:1007D000FFC4FCDD08FD0462CC67FC9308C3FFDCAA
:1007E000ED09CE0018028FDE06188F1808DF02DE32
:1007F000081AEF0418DE0218EC0904040404C3000C
:1008000001ED06FF01265FE700E7016F0B6F0ACEDF
:10081000E603E60018E70A8400C4F018ED090404B2
:10082000040418E706CEE662E6008F4F18E6068F4E
:10083000C5022717088FCE00004D2A010918CE9057
:1008400000183C18CE0001183C2019088FCE00007B
:100850004D2A0109DD04CCC97B3736DC04CC000508
:100860003736DC04BD5C9418381838FD5E61FF5ED5
:100870005FDD0A8FDD08DC0A05DE088F59498FD35A
:100880000A8FD90999088F18DE0618ED0DCDEF0BE8
:10089000FD5E5BFF5E5918EC0DD30A8FD9099908EC
:1008A0008FFD5E65FF5E6318EC0D05FD5E5518EC6F
:1008B0000B5949FD5E5307843F84BF067F5E587F16
:1008C0005E577F5E5EBD0849BD3F02F67001C511EF
:1008D0002707CEE248C685E700CEE20EC602E70053
:1008E000F67000C1FF271A5D261018DE064F5F184C
:1008F000ED03CC020018ED012007CEE249C691E7D6
:100900000018CEE208DE06EC03EE018AE7CA018F8A
:100910008A58CAB08FBD5D6318ED02CDEF0018ECA8
:1009200002FD046018EC00FD045E188FF6045318F5
:100930008F18DF0A7F000A7F00097F0008DC0ADECB
:100940000818CE0004BD5CF4D30A8FD90999088F2A
:10095000DD0ADF08BD052ECE00004F18CE0008BD11
:100960005CF4D30A8FD90999088FDD0ADF08BD0529
:100970002ECE00004F18CE000CBD5CF4D30A8FD9E8
:100980000999088FDD0ADF08BD052ECE00004FDD76
:100990000C7F000F7F000EDC0ADE08D30E8FD90D0E
:1009A000990C8FDD0ADF08BD052ECE00004F18CE52
:1009B0000015BD5CF4D30A8FD90999088FDD0ADFD1
:1009C00008BD052ECE00004F18CE001CBD5CF4D330
:1009D0000A8FD90999088FDD0ADF08BD052ECE00E0
:1009E000004F18CE001EBD5CF4D30A8FD9099908B8
:1009F0008FDF08CEE66CED02DC08ED00C601BD0716
:100A00000D0ECF20FCDE063CDE003CDE023CDE04A8
:100A10003C9F0638DF0438DF0238DF0038DF063B52
:100A2000DE063CDE003CDE023CDE043C9F06CEE2FD
:100A3000196F0007BA00800638DF0438DF0238DF9C
:100A40000038DF063BDE063C9F06CEE84C4F5FEDEC
:100A500002CC0100ED00CEE2044F5FED02CC0100BC
:100A6000ED0038DF0639DE063C9F06CEE84CCC08A8
:100A700000ED024F5FED00CEE204CC0800ED024F26
:100A80005FED0038DF0639DE063C9F06CEE84C4FAE
:100A90005FED02CC2000ED00CEE2044F5FED02CC12
:100AA0002000ED0038DF0639DE063C9F06CEE84C1C
:100AB0004F5FED02CC4000ED00CEE2044F5FED024F
:100AC000CC4000ED0038DF0639DE063C9F06CEE85C
:100AD0004C4F5FED02CC8000ED00CEE2044F5FEDA5
:100AE00002CC8000ED0038DF0639DE063C9F06CEE2
:100AF000E84C4F5FED02CC0001ED00CEE2044F5F09
:100B0000ED02CC0001ED0038DF0639DE063C9F0621
:100B1000CEE84C4F5FED02CC0002ED00CEE2044F78
:100B20005FED02CC0002ED0038DF0639DE063C9FA7
:100B300006CEE84C4F5FED02CC0004ED00CEE2049F
:100B40004F5FED02CC0004ED0038DF0639DE063CD5
:100B50009F06CEE84C4F5FED02CC0008ED00CEE2E0
:100B6000044F5FED02CC0008ED0038DF0639DE06E9
:100B70003C9F06CEE84C4F5FED02CC0040ED00CE2E
:100B8000E2044F5FED02CC0040ED0038DF0639DEB5
:100B9000063C349F06DE083CDE0A3CCEE84C4F5F44
:100BA000ED02CC0080ED00CEE244E600F7046427BD
:100BB0001ACEE847E700C601373418CE0000183CCB
:100BC000183CCC0083BD3F36383838F6046418DE54
:100BD0000618E7014F1A83005E23037E0FC405C386
:100BE0005D80188FCDEE006E00CEE246C602E700B3
:100BF000CEE2044F5FED02CC0080ED00BD15557EC6
:100C00000FCBF65E5DCEE246E700CEE2044F5FED2D
:100C100002CC0080ED007E0FCBCEE246C6FFE7009F
:100C2000CEE2044F5FED02CC0080ED00BD132B7EC1
:100C30000FCBCEE246C604E700CEE2044F5FED02E2
:100C4000CC0080ED00BD13477E0FCBCEE246C6053B
:100C5000E700CEE2044F5FED02CC0080ED00BD1353
:100C6000B67E0FCBCEE246C606E700CEE2044F5F6B
:100C7000ED02CC0080ED00BD1A2EBD33A0BD33A027
:100C8000BD33A0BD33A0BD33A0BD33A0BD33A07E16
:100C90000FCBCEE246C609E700CEE2044F5FED027D
:100CA000CC0080ED00BD13DD7E0FCBCEE246C60A40
:100CB000E700CEE2044F5FED02CC0080ED00BD13F3
:100CC000637E0FCBCEE208EC02FD0460EC00FD0475
:100CD0005ECCFFFFED02CCFF7F200BCEE208FC04D0
:100CE00060ED02FC045EED00CEE245C6017E0FC958
:100CF000BD0615200B18DE0618E601CBEDBD07EE8C
:100D0000CEE2457E0FC97F0458BD068320DA18DE87
:100D10000618E601CBBEBD082720E5F67000C1FF2E
:100D200027C65D2605BD41FA20BEBD429220B9BD51
:100D3000081720CCBD05E420C7BD05FD20C24F5FCC
:100D4000FD014EFD014CFD0152FD0150FD0156FD1E
:100D50000154FD015AFD0158208E7F0457C6023709
:100D60003418CE7740183CCC72E820107F0457C668
:100D700001373418CE76C0183CCC70B8BD0785CE8C
:100D8000E245E70038387E0FCB7F0457BD488E7EA2
:100D90000DE87F0457BD489C7E0DE8CEE2044F5F0E
:100DA000ED02CC0080ED00FE0462E60127066F0B29
:100DB0006F0A6F01FE0462C601E7002058CEE2040C
:100DC0004F5FED02CC0080ED00FE04626F007E0DEF
:100DD000E8CEE2044F5FED02CC0080ED00BD58E2AA
:100DE0007E0DE8CEE2044F5FED02CC0080ED00BD49
:100DF0005B747E0DE8CEE2044F5FED02CC0080ED27
:100E000000FE0462E60027066F0B6F0A6F00FE0407
:100E100062C601E701FE04626F096F087E0E00CE14
:100E2000E2044F5FED02CC0080ED00FE04626F0132
:100E30007E0DE8CEE2044F5FED02CC0080ED00FCB9
:100E4000769EDD0AFC769CDD08DC0ADE088A00CA94
:100E500001201ECEE2044F5FED02CC0080ED00FCCD
:100E6000769EDD0AFC769CDD08DC0ADE0884FFC481
:100E7000FEFD769EFF769C7E0DE8CEE2044F5FED90
:100E800002CC0080ED00BD28F47E0DE8CEE2044FD8
:100E90005FED02CC0080ED00BD29207E0DE8CEE2A2
:100EA000044F5FED02CC0080ED007F045D7E0DE815
:100EB000CEE2044F5FED02CC0080ED00C601F704E6
:100EC0005D7E0E00CEE245C6FEE700CEE2044F5F37
:100ED000ED02CC0080ED0038DF0A38DF083138DF62
:100EE0000639DE063C9F06CEE84CCC0100ED024FF1
:100EF0005FED00CEE204CC0100ED024F5FED00BDDE
:100F0000274838DF0639DE063C349F06DE083CDE23
:100F10000A3CCEE84CCC8000ED024F5FED00CEE203
:100F200004CC8000ED024F5FED00F65E5718DE0640
:100F300018E701CEE246CA30E70018E6015CF75E2A
:100F400057C109261C18CEE20818EC02DD0A18EC7D
:100F500000DD08DC0ADE088A80CA0018ED02CDEF49
:100F60000038DF0A38DF083138DF0639DE063C9FFB
:100F700006CEE84CCC0200ED024F5FED00CEE2045D
:100F8000CC0200ED024F5FED00F65E5ECEE246E77A
:100F9000005CF75E5E38DF0639DE063C9F06CEE673
:100FA0003FE600C5012750CEE801E6004F1A830056
:100FB0000627232E081A8300042710203A1A8300DC
:100FC00008271E1A83000A2723202CCEE800C60417
:100FD000E700C605201FCEE800C606E700C60720CA
:100FE00014CEE800C608E700C6092009CEE800C60E
:100FF0000AE700C60BE700CEE204CC0400ED024F86
:101000005FED00CEE84CCC0400ED024F5FED003800
:10101000DF0639DE063C9F06CEE84CCC1000ED0220
:101020004F5FED00CEE204CC1000ED024F5FED000B
:1010300038DF0639DE063C9F06CEE84CCC4000ED9A
:10104000024F5FED00CEE204CC4000ED024F5FEDB9
:1010500000CEE246C6AEE70038DF0639DE063C9F2A
:1010600006CEE84CCC0001ED024F5FED00CEE26809
:10107000E600F7046553CEE269E700CEE204CC0057
:1010800001ED024F5FED0038DF0639DE063CDE0081
:101090003CDE023CDE043C9F06DE083CDE0A3CDE11
:1010A0000C3CDE0E3CCEE208EC02DD0AEC00DD0872
:1010B000CEE204EC02DD0EEC00DD0CDC0ADE08BD45
:1010C0005D63940ED40F8F940CD40D8FDD0EDF0C66
:1010D0004F5F8F8410C4008F8C00002604DD002732
:1010E00003BD43ACCEE208EC02DD0AEC00DD08DC17
:1010F0000ADE08BD5D63940ED40F8F940CD40D8F5F
:10110000DD0EDF0C4F5F8F8402C4008F8C00002641
:1011100004DD002703BD41B5DE0C4F5F8F8408C49A
:10112000008F8C00002604DD002703BD4215DC0E75
:101130008404C400CE00002604DD002703BD1099FE
:10114000DC0E8401C400CE00002604DD002703BDB0
:101150000FE2DC0E85802703BD1006DC0E8402C47E
:1011600000CE00002604DD002703BD106CDE0C4F0E
:101170005F8F8400C4108F8C00002604DD002703DD
:10118000BD33A0DE0C4F5F8F8400C4208F8C000025
:101190002604DD002703BD33FFDE0C4F5F8F844044
:1011A000C4008F8C00002604DD002703BD0BA8DEE1
:1011B0000C4F5F8F8404C4008F8C00002604DD0078
:1011C0002703BD14BDDC0E8420C400CE000026041D
:1011D000DD002703BD4FE9DC0E8440C400CE0000D3
:1011E0002604DD002703BD1134DC0EC5012703BD35
:1011F000115CDE0C4F5F8F8400C4808F8C00002652
:1012000004DD002703BD0C8FCEE244E6002703BDBA
:101210000C8F38DF0E38DF0C38DF0A38DF0838DF94
:101220000438DF0238DF0038DF063BDE063C9F066D
:10123000CEE234CC0064ED024F5FED00CEE23CC65E
:1012400002E70038DF0639DE063C9F06CEE238CCE6
:101250000032ED024F5FED00CEE23CC610E70038F1
:10126000DF0639DE063C9F06DE083CDE0A3CDE0C6B
:101270003CDE0E3C7F000F7F000E7F000D7F000CD8
:10128000CEE84CDC0EED02DC0CED00CEE244E600D4
:101290007F000AD70B7F00097F0008CEE848DC0AF0
:1012A000ED02DC08ED00DC0EDE0CC30001240108B9
:1012B000DD0EDF0C20CADE063C9F06CC0010373660
:1012C0004F5F3736CC0180BD416BCC0180BD419E64
:1012D000CEE246C6AAE700383838DF0639DE063CDB
:1012E0003C9F06DE083CDE0A3CDE0C3CDE0E3CCCBD
:1012F0000212BD419EDD0EDF0CC41F18DE0618E78A
:1013000001DC0E8400C460CE000018CE0005BD5D77
:101310000718DE0618E702DC0EDE0C18CE0007BD4B
:101320005D078C000026061A83000127358C00001B
:1013300026061A83000125188C000026061A830051
:101340000227348C000026581A830003273B2050C4
:10135000DE064FE602050505050505EA01CEE24871
:10136000203A18DE064F18E60205050505050518A2
:10137000EA01CEE2492025DE064FE6020505050515
:101380000505EA01CEE24A201318DE064F18E602F0
:1013900005050505050518EA01CEE24BCA20E70060
:1013A000CEE8484F5FED02CC0800ED0038DF0E3884
:1013B000DF0C38DF0A38DF083838DF0639DE063C54
:1013C0009F0638DF0639DE063C9F06DE083CDE0A53
:1013D0003C188FDE06EC07DD0AEC05DD08CEE222C4
:1013E0001AEF00CEE228DC0AED02DC08ED00CEE2C6
:1013F0002118DE0618E60AE700CEE210C601E70073
:10140000CEE220C603E700CEE210E600C50127F7D2
:10141000C601E70038DF0A38DF0838DF0639DE06A4
:101420003C9F06CEE222ED00CEE221C60FE700CEC1
:10143000E210C601E700CEE220E700CEE210E600AF
:10144000C50127F7C601E700CEE224EC02EE001842
:101450003818DF0639DE063C3C9F06DE083CDE0A13
:101460003CDE0C3CDE0E3C7F000F7F000E7F000D4B
:101470007F000CCC0208DE06ED01DC0E05DE0C8FD1
:1014800059498FC30001240108DD0EDF0CC60F3758
:101490003418DE0E183C18DE0C183CDE06EC01BDDC
:1014A00014C6383838DE061AEE0118081AEF01188B
:1014B0008C021323C57F000F7F000E7F000D7F007D
:1014C0000CCE020818DE06CDEF0118DE0618EC017E
:1014D000BD151EDD0ADF08DC0E05DE0C8F59498FB5
:1014E000C30001240108DD0EDF0CDE089C0C26077A
:1014F000DC0A1A930E2707CEE246C6FFE70018DE85
:1015000006CDEE0108CDEF018C021323BDCEE246DD
:10151000C6AAE70038DF0E38DF0C38DF0A38DF08EC
:101520003838DF0639DE063C9F06CEE60FE600546B
:101530004FC401CE00002604DD0027EE38DF063957
:10154000DE063C9F06DE083CDE0A3C18CEE60018AC
:10155000EC02DD0A18EC00DD08DC0ADE0884FFC4BA
:10156000FE18ED02CDEF0018CEE61018EC02DD0AF1
:1015700018EC00DD08DC0ADE0884FFC4FE18ED026A
:10158000CDEF0038DF0A38DF0838DF0639DE063CE9
:101590009F06DE083CDE0A3CDE0C3CDE0E3CDD0035
:1015A000270B4F5FDD0ECC0080DD0C200C7F000F81
:1015B0007F000E7F000D7F000C18CEE60418EC02B1
:1015C000DD0A18EC00DD08DC0ADE088F84FFC47F2A
:1015D0008F9A0EDA0F8F9A0CDA0D8F18ED02CDEF7D
:1015E0000038DF0E38DF0C38DF0A38DF0838DF0656
:1015F00039DE063C9F06DE083CDE0A3CDE0C3CDEA3
:101600000E3CDD00270B4F5FDD0ECC0100DD0C2012
:101610000C7F000F7F000E7F000D7F000C18CEE6C0
:101620000418EC02DD0A18EC00DD08DC0ADE088F85
:1016300084FEC4FF8F9A0EDA0F8F9A0CDA0D8F1882
:10164000ED02CDEF0038DF0E38DF0C38DF0A38DF6F
:101650000838DF063918DE06183C9F0618DE081821
:101660003C18DE0A183C18DE0C183C18DE0E183C3C
:101670008F8403C4FF8FDD0EDF0C18CEE60818EC54
:1016800002CDEE004F5F8F84FCC4008FDD0ADF08BF
:10169000DC0EDE0C9A0ADA0B8F9A08DA098F18ED45
:1016A00002CDEF00CEE604EC02DD0AEC00DD08DC42
:1016B0000ADE088F8A02CA008FDF08CEE604ED0238
:1016C000DC08ED00BD1625CEE604EC02DD0AEC00D8
:1016D000DD08DC0ADE088F84FDC4FF8FDF08CEE65C
:1016E00004ED02DC08ED0038DF0E38DF0C38DF0ACD
:1016F00038DF0838DF0639DE063C9F06CC0001BD26
:10170000168DBD16254F5FBD168D38DF063918DEE4
:1017100006183C9F0618DE08183C18DE0A183C180C
:10172000DE0C183C18DE0E183C8401C4FFCE00000D
:10173000DD0EDF0C18CEE60418EC02DD0A18EC0012
:10174000DD08DC0ADE0884FEC400DD0ADC0EDE0CE7
:101750009A0ADA0B8F9A08DA098F18ED02CDEF009A
:1017600018EC02DD0A18EC00DD08DC0ADE088F8ABE
:1017700004CA008F18ED02CDEF00BD162518CEE685
:101780000418EC02DD0A18EC00DD08DC0ADE088F24
:1017900084FBC4FF8F18ED02CDEF0038DF0E38DF79
:1017A0000C38DF0A38DF0838DF063918DE06183C47
:1017B0003C3C9F0618DE08183C18DE0A183C18DE70
:1017C0000C183C18DE0E183CDD0A18DE0618EC0B6F
:1017D000DD0E18EC09DD0CDC0A18CE0004BD5CF44B
:1017E0008403C4F0CE000018DE0618ED03CDEF012F
:1017F00018DF0218CEE60018EC02DD0A18EC00DD56
:1018000008DC0ADE0884FCC40F18DF0418DE0218A6
:10181000AA0318EA048F18AA0118EA028F18DE0436
:1018200018ED02CDEF00DC0EDE0C8F8403C4FF8FB9
:1018300018DE0218ED03CDEF0118CEE60818EC0211
:10184000CDEE004F5F8F84FCC4008F18DF0418DEDC
:101850000218AA0318EA048F18AA0118EA028F18BE
:10186000DE0418ED02CDEF0038DF0E38DF0C38DF74
:101870000A38DF08383838DF063918DE06183C9F8A
:101880000618DE08183C18DE0A183C18DE0C183C56
:1018900018DE0E183C8C00002604DD00270BCC005F
:1018A00008DD0E4F5FDD0C200C7F000F7F000E7FE8
:1018B000000D7F000C18CEE60018EC02DD0A18ECD3
:1018C00000DD08DC0ADE0884FFC4F79A0EDA0F8F09
:1018D0009A0CDA0D8F18ED02CDEF00CEE604EC0283
:1018E000DD0AEC00DD08DC0ADE088F8A00CA808F82
:1018F000DF08CEE604ED02DC08ED00BD1625CEE6DD
:1019000004EC02DD0AEC00DD08DC0ADE088F84FF4F
:10191000C47F8FDF08CEE604ED02DC08ED0038DF7F
:101920000E38DF0C38DF0A38DF0838DF0639DE060C
:101930003C9F06DE083CDE0A3CDE0C3CDE0E3CBD75
:1019400016404F5FBD17F7CC0001CE0000BD180E4A
:10195000C6FF18CEE24618E700CC0002CE0000BD5C
:10196000180EC6FE18CEE24618E700CC0004CE00E2
:1019700000BD180EC6FD18CEE24618E700CC0008E0
:10198000CE0000BD180EC6FC18CEE24618E700CC0B
:101990000040CE0000BD180EC6FB18CEE24618E788
:1019A00000CC0080CE0000BD180EC6FA18CEE2466C
:1019B00018E7007F000B7F000A7F00097F0008CC3A
:1019C0000001CE0000BD180ECC0001CE0000BD19F4
:1019D0007ADE0A3C3CCCC0003736CC00053736CC2A
:1019E0000001BD18ABCC0001BD16F1BD16254F5F3F
:1019F000BD16F1DC0ADE08BD197ACC0002CE00006B
:101A0000BD180EC6F818CEE24618E700CC0001CE8D
:101A10000000BD180ECC0001CE0000BD197ACC002C
:101A200001BD16F1BD16254F5FBD16F1BD1625DCB3
:101A30000ADE08BD197ABD1625CC0002CE0000BD15
:101A4000180ECC0001CE0000BD180E3838383818FA
:101A5000CEE610DC0EDE0CBD5D63DD0ADF0818EC9F
:101A600002CDEE00940AD40B8F9408D4098F18EDA0
:101A700002CDEF00BD1625CC0002CE0000BD180E31
:101A8000CC0001BD17F7CC0001BD168DBD16254F4A
:101A90005FBD168DC6F618CEE24618E700CC0001F1
:101AA000BD168DBD16254F5FBD168DC6F518CEE24D
:101AB0004618E70038DF0E38DF0C38DF0A38DF0859
:101AC00038DF0639DE063C9F06CEE60FE600C4028C
:101AD00027F738DF0639DE063C9F06C601CEE6044E
:101AE000E7008DE0CEE6046F0038DF0639DE063C05
:101AF0009F06CEE607E700C604CEE604E7008DC4E5
:101B0000CEE6046F0038DF0639DE063C9F06DE08AD
:101B10003CDE0A3CCEE604EC02DD0AEC00DD08DC2B
:101B20000ADE088F8A00CA808FDF08CEE604ED0245
:101B3000DC08ED008D8ECEE604EC02DD0AEC00DD63
:101B400008DC0ADE088F84FFC47F8FDF08CEE6043E
:101B5000ED02DC08ED0038DF0A38DF0838DF06392F
:101B6000DE063C3C9F06CEE603585858C40818DEF3
:101B70000618E702E600C4F718E70118E60218EABB
:101B800001E7008D843838DF0639DE063C3C9F06CD
:101B9000CEE6131C0001CEE603585858C40818DEE0
:101BA0000618E702E600C4F718E70118E60218EA8B
:101BB00001E700CEE6061C0008FC017EFE017CBDAC
:101BC00048AA18CEE60F18E600C5012609CEE2069F
:101BD000E600C50227EC18E600C50127035F2002D6
:101BE000C601CEE6061D0008CEE6131D00014F38E3
:101BF00038DF0639DE063C9F06CEE6031C0001CC2A
:101C00000006CE0000BD48F6CEE6031D000138DF19
:101C10000639DE063C3C3C3C9F06DE083CDE0A3CC6
:101C2000DE0C3CDE0E3CBD053BCE00004F18CE0066
:101C300015BD5CF44F5F8F8403C4E08FDD0EDF0CB5
:101C400018CEE66C18EC02DD0A18EC00DD08DC0AA0
:101C5000DE088F84FCC41F8FDF08DC0EDE0C9A0ABE
:101C6000DA0B8F9A08DA098F18ED02CDEF00C60162
:101C7000BD1BED18DE06186F01CEE603E600C503B6
:101C80002620FC0196FE01942604DD00270FC60FD6
:101C9000BD1C8ADF04DE06E701DE042005C60FBD99
:101CA0001C60DE066D0127037E1F7018FE045A18A3
:101CB000EC12DD0A18EC10DD08DC0ADE088403C42F
:101CC000F08F8407C4F08FDD0EDF0C18DF0418CE10
:101CD000E60018EC02DD0A18EC00DD08DC0ADE087C
:101CE00084FCC40F8F84F8C40F8FDD0ADF08DC0E7C
:101CF000DE0C9A0ADA0B8F9A08DA098F18ED02CDFA
:101D0000EF0018DE0418EC128400C402CE0000DDDF
:101D10000EDF0C18CEE60018EC02DD0A18EC00DD30
:101D200008DC0ADE0884FFC4FDDD0ADC0EDE0C9A46
:101D30000ADA0B8F9A08DA098F18ED02CDEF00FC52
:101D400001A6FE01A4BD48F618FE045A18EC128440
:101D500000C401CE0000DD0E18DF0418CEE6001826
:101D6000EC02DD0A18EC00DD08DC0ADE0884FFC4A2
:101D7000FEDD0ADC0EDE0C9A0ADA0B8F9A08DA090D
:101D80008F18ED02CDEF0018DE0418EC16DD0A18EE
:101D9000EC14DD0818CEE604DC0ADE0884F0C4008A
:101DA0008F8400C43F8FDD0EDF0C18EC02DD0A18B3
:101DB000EC00DD08DC0ADE08840FC4FF8F84FFC45A
:101DC000C08FDD0ADF08DC0EDE0C9A0ADA0B8F9A70
:101DD00008DA098F18ED02CDEF0018DE04CEE60810
:101DE00018EC1AED0218EC18ED0018EC1ADD0A18C0
:101DF000EC18DD08DE088F8403C4FF8F18CEE8518D
:101E000018E600C4013734DC0ABD1FC118FE045AAD
:101E1000CEE79018EC1EED0218EC1CED00CEE79416
:101E200018EC22ED0218EC20ED00BD1BD6CEE60327
:101E3000E60018DE0618E7068400C40318ED023138
:101E4000312625FC0196FE01942604DD0027131897
:101E5000DE0618E603BD1C8ADF04DE06E701DE04A9
:101E6000200618E603BD1C6018DE06186D01270465
:101E70004F5F203AFE045AE617BD1BEDBD053BC47B
:101E80001FDE06E70518CEE66D18E600C4E0E7049D
:101E9000E605EA0418E700FC045AC30010CE001857
:101EA0003C3736CC02ECBD5C63CC0001383838DFFF
:101EB0000E38DF0C38DF0A38DF0838383838DF06EC
:101EC0003918DE06183C3C3C3C9F0618DE08183CDE
:101ED00018DE0A183C18DE0C183C18DE0618ED0453
:101EE000CDEF027F000DFC5E5BDD0AFC5E59CDA3E9
:101EF0000225092246DC0ACDA304223FFC5E65DDF3
:101F00000AFC5E6318DE06CDA30225092225DC0A41
:101F1000CDA304221EFC5E55DD0AFC5E5318DE06CE
:101F2000CDA302250E2207DC0ACDA30423057F00E2
:101F30000D2008188FC601D70D188FD60D18DE0694
:101F400018E10C2716CEE8515818E706E600C4FD44
:101F500018E70118E60618EA01E7004FD60D38DF4A
:101F60000C38DF0A38DF0838383838DF0639DE0643
:101F70003C9F06CEE6041C0002BD1BC4CEE6041D39
:101F8000000238DF0639DE063C308FC3FFE78F35AD
:101F90009F06DE083CDE0A3CDE0C3CDE0E3CBD0546
:101FA0003BCE00004F18CE0015BD5CF44F5F8F8410
:101FB00003C4E08FDD0EDF0C18CEE66C18EC02DDFA
:101FC0000A18EC00DD08DC0ADE088F84FCC41F8FD1
:101FD000DF08DC0EDE0C9A0ADA0B8F9A08DA098F1A
:101FE00018ED02CDEF00F60454D709F60453D109D9
:101FF000240CD701DE008F4F8FCC00012011188FE9
:10200000D609188F8F18DF00D6014F8FCC0010BD76
:102010005D6ACE00004D2A010918DE0618ED12CDCA
:10202000EF10FC01A2DD0AFC01A0DD08DC0ADE08DD
:1020300018A41218E4138F18A41018E4118F8C0040
:10204000002604DD00272B18CE0008183C18CE000F
:1020500000183CCC000837367F00037F0002DC020A
:1020600037363734BD4CEF1830188FC3000A188F3D
:10207000183518CEE60018EC02CDEE004F5F8F84C5
:1020800007C4F08F18CE0014BD5D07D70DC107221D
:1020900056CE00013A8FCE000018CE0014BD5CF47D
:1020A0004F5F8F8407C4F08F18DE0618ED17CDEF51
:1020B0001518DF0218CEE60018EC02DD0A18EC0055
:1020C000DD08DC0ADE088F84F8C40F8FDF08DE022B
:1020D0004F5FEE159A0ADA0B8F9A08DA098F18ED1E
:1020E00002CDEF00BD1C0918CEE79018EC02DD0A06
:1020F00018EC00DC0A8400C40ECE000018ED02CDFE
:10210000EF0018CEE79418EC02CDEE004F5F8F84FD
:10211000FCC4008F18ED02CDEF00D60DC107224A96
:10212000CE00004FD60D18CE0014BD5CF44F5F8F6B
:102130008407C4F08FDD0EDF0C18CEE60018EC0229
:10214000DD0A18EC00DD08DC0ADE088F84F8C40F15
:102150008FDF08DC0EDE0C9A0ADA0B8F9A08DA0998
:102160008F18ED02CDEF00BD1C09BD206ECEE60834
:10217000EC02DD0EEC00DD0C18FE045A18EC1ADD42
:102180000A18EC18DD08DC0ADE088F8403C4FF8F10
:1021900018DF0218DE0618ED03CDEF01DE0C4F5FED
:1021A0008F8410C4008F18ED0BCDEF09DC0EDE0C10
:1021B0008F8403C4FF8FDF0C84C0C4008F8403C4EA
:1021C000FF8F18ED07CDEF05DE02EE104F5F8F8415
:1021D00007C4F08F18CE0014BD5D07DE06E70E18A9
:1021E000CEE60018EC0218EC00DF028F4F5F8F8400
:1021F00007C4F08F18CE0014BD5D0718DF0418DE89
:102200000218E70DCEE851E600C40118E70F18E602
:102210000D18DE043CDE02E10E38247518DE0618C7
:102220006C0DCE00004F18E60D18CE0014BD5CF406
:1022300018CEE6004F5F8F8407C4F08F18DF0418B4
:10224000DE0618ED17CDEF1518DF0218DE0418ECC6
:1022500002DD0A18EC00DD08DC0ADE088F84F8C411
:102260000F8FDF08DE024F5FEE159A0ADA0B8F9AA6
:1022700008DA098F18ED02CDEF00BD1C09CC00046F
:10228000CE0000BD48F618DE0618E60D18E10E2552
:102290008BDC0C18DE06CDA30123037E2430250A37
:1022A000DC0ECDA30325037E243018DE0618EC07D0
:1022B000CDEE05C32000240108DD0EDF0CDC0CCDC3
:1022C000A301250F23037E24ABDC0ECDA30325033E
:1022D0007E24ABDC0EDE0C18DE0618AA0B18EA0C06
:1022E0008F18AA0918EA0A8F18CEE60818ED02CD51
:1022F000EF0018DE0618E60F3734DC0EDE0CBD1FCB
:10230000C1DE06E70FBD206EDC0EDE0CC32000240C
:102310000108DD0EDF0C3131DC0C18DE06CDA30127
:1023200025B123037E24ABDC0ECDA30325A5207BA2
:1023300018DE0618EC07CDEE05832000240109DD28
:102340000EDF0CDC0CCDA3012209255FDC0ECDA332
:10235000032358DC0EDE0C18DE0618AA0B18EA0C54
:102360008F18AA0918EA0A8F18CEE60818ED02CDD0
:10237000EF0018DE0618E60F3734DC0EDE0CBD1F4A
:10238000C1DE06E70FBD206EDC0EDE0C83200024CC
:102390000109DD0EDF0C3131DC0C18DE06CDA301A6
:1023A00022B12507DC0ECDA30322A818FE045ACEC5
:1023B000E60818EC1AED0218EC18ED0018DE061805
:1023C000E60F373418EC03CDEE01BD1FC1BD206E02
:1023D000CEE600EC02EE004F5F8F8407C4F08F184A
:1023E000CE0014BD5D07DF04DE06E70D3131DF02EC
:1023F000DE043CDE02E10E38236518DE06186A0DA5
:10240000CE00004F18E60D18CE0014BD5CF418CEB7
:10241000E6004F5F8F8407C4F08FDD0EDF0C18ECF1
:1024200002DD0A18EC00DD08DC0ADE088F84F8C43F
:102430000F8FDF08DC0EDE0C9A0ADA0B8F9A08DAAF
:10244000098F18ED02CDEF00BD1C09CC0004CE00B1
:1024500000BD48F618DE0618E60D18E10E229B189E
:10246000FE045A18EC1EDD0A18EC1CDD08DC0ADE3E
:102470000884FFC4FE18DF0418CEE79018ED02CDE3
:10248000EF0018DE04CEE79418EC22ED0218EC20E1
:10249000ED00BD206EFE045A18CEE790EC1E18ED3C
:1024A00002EC1C18ED00BD206EFC01A2DD0AFC014F
:1024B000A0DD08DC0ADE0818DE0618A41218E413F2
:1024C0008F18A41018E4118F8C00002604DD00275B
:1024D00020CC000837367F00037F0002DC0237364D
:1024E000CE00003C3C3734BD4CEF308FC3000A8F28
:1024F00035BD053BC41FDE06E71918CEE66D18E6AC
:1025000000C4E0E714E619EA1418E700FC045AC313
:102510000010CE00183C3736CC02ECBD5C63383876
:1025200038DF0E38DF0C38DF0A38DF08308FC300A1
:10253000198F3538DF0639DE063C349F06DE083C4D
:10254000DE0A3CDE066F01FC0196FE0194260FDDDB
:102550000027132009BD1CF4C601DE06E701BD1DDE
:10256000125D27F12003BD1D12DE066D01271EFC42
:102570000192DD0AFC0190DD08DC0ADE08C30001DF
:10258000240108DF08FD0192DC08FD019038DF0A14
:1025900038DF083138DF0639DE063C3C349F06DE82
:1025A000083CDE0A3CCE0000DF02DE06DD04DC0271
:1025B000E701DC04CEE760EC02DD0AEC00DC0A8413
:1025C00003C4FFDE02DD008FD3008F18DE06186C17
:1025D0000118E601DF02C10723DACEE72CEC02DDA9
:1025E0000AEC00DC0A843FC4E0CE000018CE0005EF
:1025F000BD5D073736381A8300FF2F2D18DE06DF42
:1026000004DE02CDEF028FDE04DD002A06C3000FD8
:1026100018ED0218DE0618EC024756475647564793
:1026200056DF00D3008BFE2013DC022A03C3000F09
:102630004756475647564756DF00D30038DF0A381B
:10264000DF08383138DF0639DE063C3C3C3C3C9F35
:1026500006DE083CDE0A3CCEE230FC01EEED02FC78
:1026600001ECED00CEE23CC601E700F601D0C1016D
:1026700027037E28E6BD2698DD02FE01E6DF0093F3
:1026800000DD0A2A064F5F930ADD0A9C022C0BDC50
:102690000A1AB301DE2C157E28E69C022E037E2842
:1026A000E6DC0A1AB301E02C037E28E618FE01E4FA
:1026B00018DF08DC0A1A93082F1C9C022C0D18DF67
:1026C00002DC02DF00D300DD02200BDF0218DF0096
:1026D0008F93008FDF02FE01D2DF08DC021A93081D
:1026E0002C1118DE06186F02186F01FE01DCDF08DE
:1026F0007E288D18FE01D4189C022F26FE01D818C2
:10270000DE06CDEF01DC08BD5D1ADD002A03C30043
:102710000F4756475647564756DD08FC01DC9308DD
:102720002069DC021AB301D62C58FC01DADE06ED72
:102730000118DF00DC009308ED05FC01D8ED07EC83
:1027400005EE07BD5D1ADD002A03C3000F4756479B
:102750005647564756DE06ED03EC01183C38BD5D82
:102760001ADD002A03C3000F4756475647564756FF
:10277000DD0818DE0618EC03930818ED05F301DCFC
:102780002009DE066F026F01FC01F0DD0818DE068D
:1027900018EC011AB301E8270FDC0A1AB301E22D85
:1027A0004518EE0118FF01E8FC01E8DE02BD5D1AE4
:1027B000DD002A03C3000F4756475647564756D3F6
:1027C00008FE01DCDF001A93002D0AFE01F0DF0095
:1027D0001A93002F018FFD01EAF601EBCEE76FE7B8
:1027E00000DC02FD01E638DF0A38DF083838383807
:1027F00038DF0639DE063C9F06C601F701D0BD264C
:10280000988FFC01DE05F301DE2A03C30001475661
:10281000DD008F93008FFF01E6BD274838DF0639C2
:10282000DE063C9F067F01D038DF0639DE063C3CE1
:102830003C349F06DE083CDE0A3CDE0C3CDE06E74C
:10284000014FE60B050505050505C3755CDD0C6F3D
:10285000025FF17518247F18DE0618E602186F046F
:1028600018E7055C18E70318E601270A18EC0405C9
:1028700005C3751E200818EC040505C3751C188FC8
:10288000CDEE0018DE064F18E6020505DF04DE0C6B
:10289000DD008FD3008FEC02DD0AEC00DE04DD08E2
:1028A0008FCE000018CE0006BD5CF48A00CA0F3738
:1028B000363CCC096FBD4078DE0A3CDE083CCC0AD1
:1028C00021BD40783838383818DE0618E60318E796
:1028D00002F17518258138DF0C38DF0A38DF083837
:1028E000383138DF0639DE063C9F06CEE61E1D0075
:1028F0000118FE045ACEE62418EC2AED0218EC2842
:10290000ED00CEE62818EC2EED0218EC2CED00CEF2
:10291000E62C18EC32ED0218EC30ED00CEE6301863
:10292000EC36ED0218EC34ED0038DF0639DE063CFB
:102930009F06DE083CDE0A3CDE0C3CDE0E3CCEE6AA
:102940001C1D000218FE045ACEE85C18EC42ED0291
:1029500018EC40ED00CEE86018EC46ED0218EC44AF
:10296000ED00CEE61E1D00081C0040CEE64818EC27
:102970003ADD0A18EC38DD08DC0ADF02DE0884FFE5
:10298000C41F8F8400C4FF8FDD0EDF0C18DF041816
:10299000DE0218EC02DD0A18EC00DD08DC0ADE08B5
:1029A0008400C4E08F84FFC4008FDD0ADF08DC0EE2
:1029B000DE0C9A0ADA0B8F9A08DA098F18ED02CD2D
:1029C000EF0018DE04CE00004F18E63C18CEE64CAF
:1029D00018E700CEE61DE600C50127F7CEE61E1C6F
:1029E000000838DF0E38DF0C38DF0A38DF0838DF40
:1029F0000639DE063C3C9F06CEE61E1C00011D008B
:102A000040BD053BC40FDE06E70218CEE66E18E6B1
:102A100000C4F0E701E602EA0118E700FC045AC32B
:102A20000028CE00243C3736CC0304BD5C63383824
:102A30003838DF0639DE063C308FC3FFDE8F359F26
:102A400006DE083CDE0A3CDE0C3CDE0E3CCC0A997D
:102A5000BD4103C408DE06E707BD053B585858587A
:102A600018DE0618E72018CEE66E18E600C40F1828
:102A7000DE0618E71A18E62018EA1ACEE66EE70016
:102A8000BD29E6F602DD2607FE045AE6012734FCDE
:102A9000019ADD0AFC0198DD08DC0ADE08C801FDA8
:102AA000019AFF0198FC019ADD0AFC0198FE045A84
:102AB000E6013734D60BBD292CFE045AE601F70295
:102AC000DD313118DE06186D0726037E2EBDFE04AB
:102AD0005AE606186F2118E72218EC2104040404B2
:102AE00018ED21C40118E70818E622C801C401182E
:102AF000E709FC019AFE01982607DD0026037E2CDB
:102B0000B418CE8BC0183C18CE0002183CCC096F0C
:102B1000BD407818381838CC0A21BD40CC8F84DFEE
:102B2000C4FF8FDD0ADF0818DE0618E608188F18C4
:102B3000DF0E7F000E7F000D7F000CDC0EDE0C1818
:102B4000CE001DBD5CF44F5F8F8420C4008FDD0E6E
:102B5000DF0CDC0ADE089A0EDA0F8F9A0CDA0D8F82
:102B6000DD0ADF08CC8BCF3736CC00023736CC09F4
:102B70006FBD40783838DE0A3CDE083CCC0A21BD07
:102B800040783838CE8C003CCE00023CCC096FBD7A
:102B900040783838CC0A21BD40CC8F84DFC4FF8F09
:102BA0009A0EDA0F8F9A0CDA0D8FDD0ADF08CC8CC3
:102BB0000F7E2D5ECEA7C03CCE00023CCC096FBD7F
:102BC00040783838CC0A21BD40CC8F84DFC4FF8FD9
:102BD000DD0ADF0818DE0618E608188F18DF0E7FFA
:102BE000000E7F000D7F000CDC0EDE0C18CE001DE9
:102BF000BD5CF44F5F8F8420C4008FDD0EDF0CDCE2
:102C00000ADE089A0EDA0F8F9A0CDA0D8FDD0ADFD2
:102C100008CCA7CF3736CC00023736CC096FBD4081
:102C2000783838DE0A3CDE083CCC0A21BD407838D2
:102C300038CEA8003CCE00023CCC096FBD407838AD
:102C400038CC0A21BD40CC8F84DFC4FF8F9A0EDAC6
:102C50000F8F9A0CDA0D8FDD0ADF08CCA80F3736FC
:102C6000CC00023736CC096FBD40783838DE0A3CDC
:102C7000DE083CCC0A21BD40783838CE89C03CCE35
:102C800000023CCC096FBD40783838CC0A21BD40E9
:102C9000CC84FFC4F718DE0618ED1ECDEF1C8F188C
:102CA000E6088FDF0E7F000E7F000D7F000CDC0E2C
:102CB000DE0C18CE0003BD5CF48400C408CE000016
:102CC000DD0ADF0818DE0618EC1ECDEE1C9A0ADAC3
:102CD0000B8F9A08DA098F18ED0CCDEF0ACE92C04F
:102CE0003CCE00023CCC096FBD40783838CC0A217C
:102CF000BD40CC84FFC4DFDD0ADF08DC0EDE0C182B
:102D0000CE0005BD5CF48400C420CE0000DD0EDCE6
:102D10000ADE089A0EDA0F8F9A0CDA0D8F18DE068B
:102D200018ED10CDEF0ECE94403CCE00023CCC0905
:102D30006FBD40783838CC0A21BD40CC84FFC4DF59
:102D40009A0EDA0F8F9A0CDA0D8F18DE0618ED1432
:102D5000CDEF12CE95C03CCE00023CCC096FBD40F9
:102D6000783838CC0A21BD40CC8F84FFC4F38FDD86
:102D70000EDF0CDE06E6098FDF0A7F000A7F0009FE
:102D80007F0008DC0ADE0818CE0012BD5CF4DD0A04
:102D9000DF08DC0EDE0C9A0ADA0B8F9A08DA098F4C
:102DA00018DE0618ED03CDEF0118E6082705CC0163
:102DB000012003CC0303DD0ECC0101DD0CFE045A1F
:102DC000E607C508272018CE8D40183C18CE000213
:102DD000183CCC096FBD40783838CC0A21BD40CCB6
:102DE0008A40CA00201ACE8D403CCE00023CCC095D
:102DF0006FBD40783838CC0A21BD40CC84BFC4FFB9
:102E000018DE0618ED18CDEF16F67001C504270D73
:102E1000FE045AE6068400C410DD002705C601182A
:102E2000DE0618E705F60454D709F60453D1092441
:102E30000CD701DE008F4F8FCC01002011188FD6E8
:102E400009188F8F18DF00D6014F8FCC1000BD5DA1
:102E50006ACE00004D2A010918DE0618ED1ECDEFDE
:102E60001C186F06FC01A2DD0AFC01A0DD0818ECAD
:102E70001E940AD40B8F9408D4098F8C000026046A
:102E8000DD002708C60118DE0618E706C60718CEBB
:102E9000E26418E700BD3B10CEE2641D000118DEBD
:102EA0000618E606271DCE00103CCE00003CCC00E4
:102EB0001037364F5F37363734BD4CEF308FC30095
:102EC0000A8F35CEE211C610E70018CEA68F183C47
:102ED00018CE0002183CCC096FBD40783838CE00BF
:102EE000043CCE00003CCC0A21BD40783838CEE20C
:102EF00011E600C51027F7C610E700CC0004CE008D
:102F000000BD4B55BD4F90FC019EFE019CBD48AAE3
:102F100018DE06186D052708CEE61E1C00042006E4
:102F2000CEE61E1D0004DE066D0726037E315BCE55
:102F3000E61EE600C4DF18DE0618E71B18E6085890
:102F400058585858C42018EA1BE700CE89CF3CCE09
:102F500000023CCC096FBD4078383818DE06CDEE53
:102F60000C3CCDEE0A3CCC0A21BD40783838CE92DC
:102F7000CF3CCE00023CCC096FBD4078383818DE1B
:102F800006CDEE103CCDEE0E3CCC0A21BD4078388B
:102F900038CE944F3CCE00023CCC096FBD4078380F
:102FA0003818DE06CDEE143CCDEE123CCC0A21BD25
:102FB0004078383818DE0618EC03DD0A18EC01DD1D
:102FC00008CE95C13CCE00023CCC096FBD4078389C
:102FD00038DE0A3CDE083CCC0A21BD40783838CEC9
:102FE000A44F3CCE00023CCC096FBD40783838CEAF
:102FF00000CE3CCE00003CCC0A21BD40783838CE13
:10300000A48F3CCE00023CCC096FBD40783838DE3E
:103010000E3CDE0C3CCC0A21BD40783838CEA44FA3
:103020003CCE00023CCC096FBD40783838CE00DE83
:103030003CCE00003CCC0A21BD40783838CEA48F6D
:103040003CCE00023CCC096FBD40783838DE0E3CE7
:10305000DE0C3CCC0A21BD40783838BD2A2DBD4A53
:1030600041BD4AE5CEE648E600C50127F7CEE206B7
:10307000E600C50227F7CEE20A1C0002CEE840FCBB
:10308000019AED02FC0198ED00FE045A188FE60645
:10309000188F18DF0E7F000E7F000D7F000CDC0EF6
:1030A000DE0C18CE0018BD5CF4DD0EDF0CFC019ABE
:1030B000DD0AFC01982604DC0A270ADC0EDE0C8AF5
:1030C00000CA062008DC0EDE0C8A00CA05DD0ADF15
:1030D00008CCA68F3736CC00023736CC096FBD40FE
:1030E000783838DE0A3CDE083CCC0A21BD4078380E
:1030F00038CE8D4F3CCE00023CCC096FBD407838B5
:103100003818DE06CDEE183CCDEE163CCC0A21BDBB
:1031100040783838CE00013CCE00003CCC082BBDB6
:1031200040783838FE045A4FE606CE000018CE002C
:1031300018BD5CF48A00CA0ADD0ADF08CEA68F3CFF
:10314000CE00023CCC096FBD40783838DE0A3CDE48
:10315000083CCC0A21BD40783838CC000ACE0000AB
:10316000BD4B55CC0A9ABD40CCCEE211C610E7004B
:10317000CEE211E600C51027F7C610E700FE045A9C
:103180004FE606CE000018CE0018BD5CF48A00CAD7
:1031900010DD0ADF08CEA68F3CCE00023CCC096FC2
:1031A000BD40783838DE0A3CDE083CCC0A21BD4000
:1031B000783838CEE61C1C0002CE00003C3CCC081F
:1031C0002BBD40783838CEE2641C000818CEE2608F
:1031D00018EC02DD0E18EC00DD0CFC01AADD0AFC87
:1031E00001A8DD08DE0C9C0825152207DC0E1A93C9
:1031F0000A230C18EC02FD01AA18EC00FD01A8CE70
:10320000E260EC02DD0EEC00DD0CFC01AEDD0AFC40
:1032100001ACDD0818DE0C189C0825262206DE0EFF
:103220009C0A231EFC01B2DD0AFC01B0DD08DC0AA9
:10323000DE08C30001240108DF08FD01B2DC08FD3F
:1032400001B018DE06186D06271ACE00103CCE001D
:10325000003C4F5F373637363734BD4CEF308FC3C5
:10326000000A8F35BD2AF2FE045AE606F702E2E6AE
:1032700007F702E3CC000138DF0E38DF0C38DF0A35
:1032800038DF08308FC300228F3538DF0639DE067D
:103290003C9F06BD29E6BD2A2DBD2AF238DF06393E
:1032A000DE063C349F06CEE84C4F5FED02CC0010AA
:1032B000ED00CEE63FE600C5012733F60457DE06F3
:1032C000E701262AF75E51F60453C10122207C5EF5
:1032D00050F65E50F10334230CBD05E4DE06E60132
:1032E000F75E502009CEE6471C00101D0010CEE20C
:1032F000044F5FED02CC0030ED003138DF0639DEDF
:10330000063C349F06CEE84C4F5FED02CC0020ED2A
:1033100000CEE63FE600C5012734F60457DE06E797
:1033200001262BF75E50F60453F1045823207C5EEF
:1033300051F65E51F10335230CBD05FDDE06E601B5
:10334000F75E512009CEE6471C00101D0010CEE2AA
:10335000044F5FED02CC0030ED003138DF0639DE7E
:10336000063C9F06DE083CDE0A3CDE0C3CDE0E3CE2
:10337000CEE647E600C50127037E355F18FE045AF6
:1033800018EC26DD0E18EC24DD0CFC0302DD0AFC33
:103390000300DD08DE0C9C08260ADC0E1A930A26C0
:1033A000037E355FDE0C9C08225E2507DC0E1A9337
:1033B0000A24558F18E6008FDF0A7F000A7F000974
:1033C0007F0008CC7E8F3736CC00023736CC096FB1
:1033D000BD40783838DE0A3CDE083CCC0A21BD40CE
:1033E000783838F602DEC101261EFE045AE60226AF
:1033F00017CEE7FFC608E700CEE211E600C50427B6
:10340000F7C604E7007F02DECEE6461D0080BD4918
:10341000BACC1E84CE0000BD48F6F67001C5082760
:1034200005BD1D122003BD2086BD49FFCEE20A1C4A
:10343000000218CEE206C60218E7001C0002F602DF
:10344000DE261CFE045AE602C1012613CEE7FFC6A3
:1034500009E700CEE211C604E700C601F702DEFE6E
:10346000045A188FE600188F18DF0A7F000A7F00C1
:10347000097F0008CE7E8F3CCE00023CCC096FBD98
:1034800040783838DE0A3CDE083CCC0A21BD407862
:103490003838FE045AEC16DD0AEC14DD0818CEE6C6
:1034A00004DC0ADF02DE0884F0C4008F8400C41F3D
:1034B0008FDD0EDF0C18EC02DD0A18EC00DD08DCF5
:1034C0000ADE08840FC4FF8F84FFC4E08FDD0ADFAB
:1034D00008DC0EDE0C9A0ADA0B8F9A08DA098F18CC
:1034E000ED02CDEF00CEE6051C0040CEE60FE60073
:1034F000C50227F7CEE6051D0040DE02E65AC501EB
:103500002706CEE6461C0080CC000138DF0E38DFEF
:103510000C38DF0A38DF0838DF0639DE063C3C3C71
:103520003C3C9F06DE083CDE0A3C18FE0462186D37
:103530000026037E37A3CEE2641C000818EC0A05BF
:1035400018E30A05050518DF00D300C3000CDE06EA
:10355000ED07CEE260DD02EC0218DF0418DE02188F
:10356000ED02EC0018ED0018DE0418EC0A0518E373
:103570000A050505DD00188FD300188FF6045418CE
:10358000E714CEE8BCEC02DD0AEC00DD0818FE040E
:103590006218EC0A0518E30A050505DD02DE0218CB
:1035A000DF008FD3008FDC0A8403ED1818EC0A05C6
:1035B00018E30A050505DD02DE0218DF008FD300DF
:1035C0008FCC03FF9408D409ED1A18EC0A0518E310
:1035D0000A050505DD0218DF00D300CEE740DD0255
:1035E000EC02EC00DD08CC07FF9408D409DE02ED04
:1035F0001CCEE744EC02DD0AEC00DD0818EC0A05FD
:1036000018E30A050505DD02DE0218DF008FD3008E
:103610008FDC0A8407ED1E18EC0A0518E30A05057D
:1036200005DD02DF04DE0218DF008FD3008FCC0738
:10363000FF9408D409ED20DE0418EC0A0518E30A0B
:1036400005050518DF00D300C3001018DE0618EDCD
:1036500001BD5BB518DE0618EE0118ED02CDEF00D6
:10366000CEE73E1C00041D00041C00021D0002FCED
:103670000462DE06ED03188F18EC08CEFFFF3C8DC8
:103680003018DE0618EE0318ED08FE046218DE0698
:10369000CDEF05EC0AEE04093C8D16DE06EE05EDD5
:1036A0000A383838DF0A38DF083838383838DF0663
:1036B00039DE063C9F06DE061AA30526044F5F206E
:1036C00003C3000138DF0639DE063C9F06DE083CF6
:1036D000DE0A3C18FE0462186D00275CCEE668EC3A
:1036E00002DD0AEC00DD0818EC0A0518E30A0505FE
:1036F0000518DF00D300DE0ADD0218DF0418DE0241
:10370000CDEF1618DE0418EC0A0518E30A050505C6
:10371000DD00188FD300188FCC00019408D409184D
:10372000E715C607CEE264E700CC0001CE0000BD7D
:1037300048F6CEE2641D000138DF0A38DF0838DFC2
:103740000639DE063C3C3C3C3C9F06DE083CDE0A7B
:103750003CDE0C3CDE0E3CCEE66FF60454C40F1883
:10376000DE0618E706E600C4F018E70218E60618B9
:10377000EA02E700FE045AE64EF1032A2510E65657
:10378000F103322509BD4C5D5D26037E3A03FE043C
:103790005AE603F102DF230BC601BD4BA35D2603EE
:1037A0007E3A0318CE7E8F183C18CE0002183CCC0F
:1037B000096FBD40783838CE00083CCE00003CCCC4
:1037C0000A21BD40783838FE045AFC0326DD0EFC81
:1037D0000324DD0CEC4ADD0AEC48DD0818DE0C1889
:1037E0009C0825112206DE0E9C0A2309BD2B355D9F
:1037F00026037E3A03CEE647E60018DE0618E70801
:103800008400C40118ED03264EFE045AEC26DD0E9A
:10381000EC24DD0CFC0302DD0AFC0300DD0818DEED
:103820000C189C082606DE0E9C0A272BF67001C594
:10383000082703BD49BABD345F18DE0618E701F654
:103840007001C5082703BD49FF18DE06186D012663
:103850000618EC037E3AB118FE045AFC0326DD0E6E
:10386000FC0324DD0C18EC4ADD0A18EC48DD08DE08
:103870000C9C08254C2207DC0E1A930A2543FC03F6
:103880001EDD0EFC031CDD0C18EC42DD0A18EC40BA
:10389000DD08DE0C9C082629DC0E1A930A2622FC81
:1038A0000322DD0EFC0320DD0C18EC46DD0A18ECCB
:1038B00044DD0818DE0C189C082606DE0E9C0A273C
:1038C00006BD2B355D273CFE045AE603F102DF24DA
:1038D00008C601BD4BA35D272A18CE7E8F183C1861
:1038E000CE0002183CCC096FBD40783838CE0009B4
:1038F0003CCE00003CCC0A21BD40783838BD4C5D40
:103900005D26054F5F7E3AB1CEE66FF604545858F7
:10391000585818DE0618E707E600C40F18E7051820
:10392000E60718EA05E700CEE6471C001018FE047B
:103930005AFC02EADD0EFC02E8DD0C18EC0EDD0A92
:1039400018EC0CDD08DE0C9C082607DC0E1A930A26
:103950002717CEE6D0DC0AED02DC08ED0018EC0EED
:10396000FD02EA18EC0CFD02E8CEE6D418EC0AEDF4
:103970000218EC08ED00CEE6471D0010CEE6EEE69C
:1039800000BD053BCEE7F3E700BD052ECEE7F2E72D
:1039900000CEE7EFC6F9E700CEE7EEC601E7006F1D
:1039A00000FE045AE658F70334E659F70335CC0015
:1039B0000138DF0E38DF0C38DF0A38DF08383838D6
:1039C0003838DF0639DE063C3C3C9F06F67003C5FE
:1039D000082735CEE208E60018DE0618E701CEE239
:1039E00004E60018E70418E6015318E70218E60495
:1039F00018E40218E704C508270ECEE24CE600C51D
:103A0000012705CC000120024F5F383838DF063926
:103A1000DE063C9F067D045C26467D045D2741FC56
:103A20000136FE0134BD48AA2007C608CEE210E7E1
:103A300000CEE210E600C508270ECEE206E600C57D
:103A40000226058D805D27E2CEE210E600C508263D
:103A50000FCEE206E600C5022606BD3AC55D27E8A0
:103A600038DF063918DE06183C3C349F0618DE089D
:103A7000183C18DE0A183C18DE0C183C18DE0E182C
:103A80003CDD0A18DE0618EC0EDD0E18EC0CDD0C21
:103A9000DC0A18A30A8F18E20918A2088FDD0ADFD2
:103AA00008CC010018E011820018ED0118CE0000CA
:103AB000DE06188FE703188FDC0A05DE088F5949E8
:103AC0008FDD0ADF08DF04DE0664016602DE049C87
:103AD0000C251F22051A930E2318DF04DE06188F0B
:103AE000E301188FDE04930E8FD20D920C8FDD0A46
:103AF000DF08DE066C03E603C10223BC188C00005D
:103B0000260418CE0001188F504F38DF0E38DF0C16
:103B100038DF0A38DF08383138DF063918DE061892
:103B20003C9F0618DE08183C18DE0A183C8C000082
:103B30002604DD00275FCC010018DE0618E00682AF
:103B400000DD0218CEE60418EC02DD0A18EC00DDF8
:103B500008DC0ADE08840FC4FF8F84FFC4E08FDD19
:103B60000ADF08DC02CE000018CE000CBD5CF48435
:103B7000F0C4008F8400C41F8F9A0ADA0B8F9A0852
:103B8000DA098F18CEE60418ED02CDEF00CEE60577
:103B90001C00202006CEE6051D0020CEE6051C00F8
:103BA00040BD1BC418CEE605181D004038DF0A389A
:103BB000DF0838DF0639DE063C3C3C9F06DE083C69
:103BC000D709F676ACD10926037E3D58D109243AAF
:103BD0004FF676AC8F4FF604E08F3CBD3DC3DE065A
:103BE000ED01E6023131D109245A3734CC0001CE3F
:103BF0000000BD3C1CDE06E602F776ACCE00004FAE
:103C0000F604E1BD48F6313120C64FF676AC8F4F51
:103C1000F604E08F3CBD3DF1DE06ED03E6043131F4
:103C2000D10923203734CC0001CE0000BD3C1CDE7E
:103C300006E604F776ACCE00004FF604E1BD48F688
:103C4000313120C6D6093734CC0001CE0000BD3C4E
:103C50001CD609F776AC313138DF08383838DF0642
:103C600039DE063C9F06F104D82338CEE63FE60055
:103C7000C501272CF60453F1045823244F050505EC
:103C800005C304888FE600BD3CB6BD05FD5FBD3CA5
:103C9000B65F37344F5FCE0000BD3C1C313120068B
:103CA000F604D8BD3CB67D76B02706BD54C67F76F7
:103CB000B038DF0639DE063C9F06F676AE8DA238B8
:103CC000DF0639DE063C3C9F06D70318DE0618E601
:103CD00008186F0118E70218EC01DE02DF00DB01B3
:103CE00089001A8300FF2303CC00FF4F3838DF061A
:103CF00039DE063C9F06DE083CDE0637E606D701C5
:103D0000DE00338FD7098FD10925074FD0098200F4
:103D100020024F5F4F38DF0838DF063918DE0618FB
:103D20003C9F0618DE08183C18DE0A183C18DE0C0A
:103D3000183C18DE0E183CDD0EDF0CFC76A2DD0A06
:103D4000FC76A0DD0818DE06CDA30922352507DCA8
:103D50000ACDA30B222CF676AC373418DE06CDEE56
:103D6000073CCDEE053CDE0E3CDE0C3CDC0ADE08FA
:103D7000BD3B64F776AEC601F776B030C60A3A3579
:103D8000206DFC76A6DD0AFC76A418DE06CDA3091C
:103D900022162507DC0ACDA30B240DF604DD3734EB
:103DA000F676ACBD3DC32042FC76AADD0AFC76A8BF
:103DB00018DE06CDA30922272507DC0ACDA30B2494
:103DC0001EFC76A6DD0AFC76A418DE06CDA3092526
:103DD0000E2207DC0ACDA30B2305F604DE2003F632
:103DE00004DF3734F676ACBD3DF13131F776AEBD48
:103DF0003DB538DF0E38DF0C38DF0A38DF0838DF32
:103E00000639DE063C9F06CE00403C18CE76C01830
:103E10003CCC0498BD5C634FF6045405050505C30E
:103E20000498CE00103C3736CC04D8BD5C633838DB
:103E3000383838DF0639DE063C9F06DE083CDE0AED
:103E40003C188FDE06EC07DD0AEC05DD08CEE22229
:103E50001AEF00CEE228DC0AED02DC08ED00CEE22B
:103E60002118DE0618E60AE700CEE210C601E700D8
:103E7000CEE220C603E700CEE210E600C50127F738
:103E8000C601E70038DF0A38DF0838DF0639DE060A
:103E90003C9F06CEE222ED00CEE22818DE0618E6B0
:103EA00006E700CEE221C608E700CEE210C601E731
:103EB00000CEE220C603E700CEE210E600C50127EF
:103EC000F7C601E70038DF0639DE063C9F06CEE282
:103ED00022ED00CEE22918DE0618E606E700CEE263
:103EE00021C604E700CEE210C601E700CEE220C6FC
:103EF00003E700CEE210E600C50127F7C601E700A0
:103F000038DF0639DE063C9F06CEE222ED00CEE227
:103F10002A18DE0618E606E700CEE221C602E70010
:103F2000CEE210C601E700CEE220C603E700CEE2F3
:103F300010E600C50127F7C601E70038DF0639DEC5
:103F4000063C9F06CEE222ED00CEE22B18DE0618DC
:103F5000E606E700CEE221C601E700CEE210E70068
:103F6000CEE220C603E700CEE210E600C50127F747
:103F7000C601E70038DF0639DE063C9F06DE083C56
:103F8000DE0A3C188FDE06EC07DD0AEC05DD08CE04
:103F9000E2221AEF00CEE228DC0AED02DC08ED0096
:103FA000CEE221C60FE700CEE210C601E700CEE266
:103FB00020C603E700CEE210E600C50127F7C601E0
:103FC000E70038DF0A38DF0838DF0639DE063C9FB5
:103FD00006CEE222ED00CEE221C60FE700CEE210CF
:103FE000C601E700CEE220E700CEE210E600C50100
:103FF00027F7C601E700CEE224EC02EE00183818DD
:10400000DF0639DE063C9F06CEE222ED00CEE2213D
:10401000C60FE700CEE210C601E700CEE220E700BF
:10402000CEE210E600C50127F7C601E700CEE22484
:10403000E6004F38DF0639DE063C9F06CEE222ED71
:1040400000CEE221C60FE700CEE210C601E700CEA7
:10405000E220E700CEE210E600C50127F7C601E73F
:1040600000CEE226E6004F38DF0639DE063C9F062A
:10407000DE083CDE0A3C188FDE06EC07DD0AEC05A4
:10408000DD08188F05058BE0188FDC0A18ED02DCBF
:104090000818ED0038DF0A38DF0838DF0639DE0699
:1040A0003C9F0605058BE0188F18EC02CDEE00183A
:1040B0003818DF0639DE063C349F06C6FFDE06E709
:1040C00001CEE84C4F5FED02CC0200ED00CEE63FA2
:1040D000E600C5042607BD0807DE06E701DE066D1B
:1040E000012B06CEE2081C0002CEE2044F5FED0277
:1040F000CC0200ED003138DF0639DE063C9F06CEEB
:10410000E2044F5FED02CC0200ED00CEE2081D009C
:104110000238DF0639DE063C9F06CEE84C4F5FEDE5
:1041200002CC0800ED00CEE24CE600C501270EF6F9
:104130007001C5102705BD432F20028D6BCEE24CC8
:10414000E600C502271CCEE63FE600C5042613BDE7
:1041500008075D2B0DCEE2491D00C0C602CEE24C21
:10416000E700CEE2044F5FED02CC0800ED0038DF3F
:104170000639DE063C9F067F0456F67001C501270E
:104180000DCEE24CC601E700CEE2481C008038DFCD
:104190000639DE063C9F06CEE24CC602E700CEE2C0
:1041A000491C008038DF0639DE063C3C349F06C6D9
:1041B000FF18DE0618E701C601F70456F67003186B
:1041C0006F0218E70318EC02C5082705C601F704BB
:1041D0005CCEE63FE600C5012730F60338C5012670
:1041E0002218DE0618EC028400C4071A8300012698
:1041F00012C601373418CE76C0183CCC70B8BD0753
:10420000853838BD0683DE06E70118DE06186D0125
:104210002B0DCEE2481D00C0CEE24CC601E700F6F1
:104220007003C50827037F045C383138DF0639DEA8
:10423000063C3C3C9F06C60118DE0618E701CEE2AC
:1042400048E60018E703C4DF18E70418E603C520B2
:10425000260CC601F7045918E604CA2020097F0479
:104260005918DE0618E60418E703CEE63FE600C557
:10427000012707BD0683DE06E70118DE06186D017B
:104280002B0FCEE24CC601E700CEE24818E603E76A
:1042900000383838DF0639DE063C9F06CEE63FE6BA
:1042A00000CEE7F4C60CE70038DF0639DE063C9F97
:1042B00006CEE84C4F5FED02CC1000ED00CEE63F9D
:1042C000E600C5012703BD46F4CEE2044F5FED02D0
:1042D000CC1000ED0038DF0639DE063C3C3C3C3CAF
:1042E0003C9F06DE083CDE0A3CDE06E701C601F71D
:1042F00004EFE6016F09E70AEE098C0006271F2E7E
:10430000088C000427147E46E5DE06EE098C0008C2
:1043100027168C000A27157E46E5C6042002C6052E
:1043200018DE0618E702200EC6062002C60718DEB1
:104330000618E702C60518E70318E70418DE061892
:10434000E601F104EE26037E46D9CDEE098C000687
:1043500026037E45C72E088C0004271E7E46D918EA
:10436000DE0618EC091A83000826037E45C71A8367
:10437000000A26037E45C77E46D918CEE64418ECCF
:1043800002DD0A18EC00DD08DC0ADE0884FDC4FF4B
:1043900018ED02CDEF0018EC02DD0A18EC00DD0884
:1043A000DC0ADE088A01CA0018ED02CDEF0018EC25
:1043B00002DD0A18EC00DD08DC0ADE0884FEC4FF1A
:1043C00018ED02CDEF00C603BD070D18CE01181879
:1043D0003CCE70B83CCC0338BD5C6318CE004018AE
:1043E0003CCE76C03CCC0498BD5C637F0454CC03C7
:1043F0003CFD045ABD053BC40F18DE0618E709183A
:10440000CEE66F18E600C4F018DE0618E70518E6D9
:104410000918EA05CEE66FE7004F5FBD4C5DC601A7
:10442000BD4BA3BD2637BD4F90BD338E7F045318BF
:10443000CE0010183CCE04983CCC04D8BD5C63BDC3
:10444000052E5858585818DE0618E70918CEE66F9A
:1044500018E600C40F18DE0618E70618E60918EA81
:1044600006CEE66FE700C601BD070D18DE0618E6AA
:1044700004373418E603BD4781DE06E602BD47C2B5
:10448000FC017AFE0178BD48F618FE045ACEE6D447
:1044900018EC0AED0218EC08ED00CEE7FFC606E7BF
:1044A0000030C60E3A35FC04ECDD0AFC04EADD08F7
:1044B0002607DC0A26037E46D9CEE208DC0AED0296
:1044C000DC08ED007E46D9FC0162FE0160BD48F6C5
:1044D00018CEE64418EC02DD0A18EC00DC0A843839
:1044E000C400CE00002604DD00271818EC02DD0A07
:1044F00018EC00DD08DC0ADE088A02CA0018ED02AA
:10450000CDEF0018DE0618E604373418E603BD4781
:1045100081CEE7FFC607E70018DE0618E602BD47B2
:10452000C23131F604EEC10427037E46D9C603BD6D
:10453000070D18CE0118183CCE71D03CCC0338BD05
:104540005C6318CE0040183CCE77003CCC0498BD8C
:104550005C637F0454CC033CFD045ABD053BC40F8F
:1045600018DE0618E70918CEE66F18E600C4F01842
:10457000DE0618E70718E60918EA07CEE66FE70037
:10458000BD2637BD4F90BD338EC601BD4BA34F5FD7
:10459000BD4C5DBD052E5858585818DE0618E70961
:1045A00018CEE66F18E600C40F18DE0618E70818E4
:1045B000E60918EA08CEE66FE7005FBD070DCEE218
:1045C00008EC02FD04ECEC00FD04EACCFBFFED027C
:1045D000CCEF7FED00383838387F04EF18DE06184E
:1045E000E601F704EE38DF0A38DF083838383838A3
:1045F00038DF0639DE063C349F06DE083CCEE7F5A0
:10460000E600D709CCFFFCDB0989001A83000822E9
:104610006805C35E3E188FCDEE006E00BD43972047
:1046200058CEE7F4C604E700C605201FCEE7F4C65F
:1046300006E700C6072014CEE7F4C608E700C6095F
:104640002009CEE7F4C60AE700C60B18DE0618E715
:1046500001CEE63FE600C502260ACEE7F418E601E1
:10466000E7002015D609BD43D9CEE7F418DE0618B9
:10467000E601E700D609F704EE38DF083138DF0637
:1046800039DE063C349F06DE083CDE06E701E6071D
:10469000D709CEE211C604E700CEE7FF18DE061800
:1046A000E601E700CEE211E600C50427F7C604E7FD
:1046B00000CEE7FEE600D10926DF38DF083138DF1B
:1046C0000639DE063C9F06DE083CDE0A3CDE0C3C7A
:1046D000DE0E3CD709C60F373418CE000F183C1831
:1046E000CE0000183CCC096FBD3F36C60718CEE29D
:1046F0006418E7003838388FD6098FDF0A7F000A40
:104700007F00097F0008CC7E8F3736CC0002373619
:10471000CC096FBD40783838DE0A3CDE083CCC0A54
:1047200021BD40783838CEE2641D0001CEE211E6AA
:1047300000C51027F7CC1F40CE0000BD48F6CEE2E2
:10474000641C000818CEE26018EC02DD0E18EC00C4
:10475000DD0CFC018EDD0AFC018CDD08DE0C9C0802
:1047600025152207DC0E1A930A230C18EC02FD0112
:104770008E18EC00FD018CCEE211C610E70038DF88
:104780000E38DF0C38DF0A38DF0838DF0639DE067E
:104790003C9F06C60ABD43D938DF0639DE063C9F7A
:1047A00006C604BD43D938DF063918DE06183C9F1B
:1047B0000618DE08183C18DE0A183CDD0ADF082659
:1047C0000DDD002609CC0001DD0A4F5FDD08CEE2D9
:1047D00034DC0AED02DC08ED00CEE23C1C0002CE27
:1047E000E206C602E700CEE20A1D000238DF0A3800
:1047F000DF0838DF063918DE06183C349F0618DE5D
:1048000008183C18DE0A183CDF087D04EF2744181E
:10481000CE0004BD5CF4DD0ADF0818DE06186F0167
:10482000CEE264C607E70018DE06186C0118E60140
:10483000C10423ECC606E700CEE264C60EE700CE54
:10484000E260EC02EE009C0825EE22361A930A255F
:10485000E7202FCEE234ED02DC08ED00CEE23C1C76
:104860000002CEE206C602E700CEE20A1D0002CE3A
:10487000E206E600C50227F7C602E700CEE20A1C00
:10488000000238DF0A38DF083138DF0639DE063C3F
:104890009F06DE083CD709CC7E803736CC00023735
:1048A00036CC096FBD40783838CC0A21BD4137D1AC
:1048B0000926F638DF0838DF0639DE063C9F06CCCD
:1048C000000437364F5F3736CC082BBD4078CC0814
:1048D0005BBD40CC8A00CA0837363CCC085BBD4083
:1048E00078CC0879BD40CC8A00CA0837363CCC0861
:1048F00079BD4078308FC3000C8F3538DF0639DE44
:10490000063C9F064F5F37363736CC082BBD4078C4
:10491000CC085BBD40CC84FFC4F737363CCC085B89
:10492000BD4078CC0879BD40CC84FFC4F737363C15
:10493000CC0879BD4078308FC3000C8F3538DF0646
:1049400039DE063C9F06DE083CDE0A3CCE7CC03CDD
:10495000CE00023CCC096FBD40783838CC0A21BD6E
:1049600040CCDD0ADF0818FE045A18E607C5012707
:1049700008DC0A8A00CA012008DC0ADE0884FFC4B9
:10498000FEDD0A18E607C5022708DC0A8A00CA020B
:104990002006DC0A84FFC4FDDD0ADF08CC7CCF37AB
:1049A00036CC00023736CC096FBD40783838DE0A85
:1049B0003CDE083CCC0A21BD40783838CE7CC03C77
:1049C000CE00023CCC096FBD40783838CC0A21BDFE
:1049D00040CC9C0826E61A930A26E138DF0A38DF25
:1049E0000838DF0639DE063C9F06DE083CDE0A3C5E
:1049F000CE74003CCE00023CCC096FBD4078383804
:104A0000CC0A21BD40CC84FFC4FEDD0ADF08FE04D1
:104A10005A4FE60704048400C401CE00009A0ADA63
:104A20000B8F9A08DA098FDD0ADF08CC740F37364E
:104A3000CC00023736CC096FBD40783838DE0A3CEE
:104A4000DE083CCC0A21BD4078383838DF0A38DF30
:104A50000838DF0639DE063C349F06DE083CDE0AF5
:104A60003CDE06E701CCA6803736CC00023736CCD8
:104A7000096FBD407818381838CC0A21BD40CC18D1
:104A8000CE0008BD5D07DD0A18DE0618E601C1FF8D
:104A90002706DC0AC50126CD38DF0A38DF083138A1
:104AA000DF0639DE063C3C9F06DE06E701FE045ABF
:104AB000E603F102DF277F5D267CCEE7F7C60DE730
:104AC00000C601DE06E702C602CEE206E700CEE23D
:104AD0000A1C0002DE06E6012709FC013AFE013845
:104AE000BD48AACEE206E600C5022620CEE211E6C7
:104AF00000C5012708C601E700DE066F02DE066D6D
:104B0000022709CEE206E600C50227E0CEE206C68D
:104B100002E700CEE20A1C0002DE06E6022709CE0A
:104B2000E7F76F004F5F2030CEE7F4C60EE700DEF8
:104B300006E602F702DFFE045AE603F102DF27155C
:104B4000C1012611CEE7F4C60CE700CEE7F76F00EF
:104B5000C601F702DFCC00013838DF0639DE063C3B
:104B60003C9F06CEE63EE600C504272DFE045AE62D
:104B70004EF1032A2723BD053B565656C4C0DE0618
:104B8000E702CEE66CE600C43FDE06E701E602EA95
:104B900001CEE66CE700BD4EA1C601BD4E32CC0091
:104BA000013838DF0639DE063C3C9F0618FE045A01
:104BB00018E605F102E12732CEE63D585858C40800
:104BC00018DF0418DE0618E702E600C4F718E7014C
:104BD00018E60218EA0118DE04E70018E605F702F5
:104BE000E1FC0142FE0140BD48F63838DF0639DEFF
:104BF000063C3C3C3C3C3C9F06DE083CDE0A3CDE7E
:104C00000C3CDE0E3CDE06E70A18DE06EC13DD0A7D
:104C1000EC11DD08F65E52E702EC17EE15BD5D63A0
:104C2000DD0EDF0C18E6105318E704DC0ADE081866
:104C3000A41718E4188F18A41518E4168F18ED0798
:104C4000CDEF0518E60A18E41018E70918E6022760
:104C500051CEE67CEC02DD0AEC00DD08DC0ADE0861
:104C6000940ED40F8F940CD40D8FDD0ADF04CEE6A2
:104C70008BE60054545418E40418E701DC0A18AA1F
:104C80000718EA08DF02DE048F18AA0518EA068F63
:104C900018CEE67818ED02CDEF00DE06E601EA094F
:104CA0002052CEE678EC02DD0AEC00DD08DC0ADEFC
:104CB00008940ED40F8F940CD40D8FDD0ADF04CE30
:104CC000E68BE60018DE0618E40418E701DC0A1893
:104CD000AA0718EA08DF02DE048F18AA0518EA06F8
:104CE0008F18CEE67C18ED02CDEF00DE06E601EA75
:104CF00009585858DE02E70018DE0618E602C80117
:104D0000F75E52CEE63F565656C4C018E70AE60094
:104D1000C43F18E70318E60A18EA03E70038DF0E75
:104D200038DF0C38DF0A38DF08383838383838DFF1
:104D30000639DE063C349F06DE06E70118FE045AFB
:104D400018E656F103322754CE70043AFC70B2379D
:104D500036FC70B037364F18E6560505DD02DF0425
:104D6000DE028FC370248FEC023736EC00DE04378E
:104D700036F670A63734E600BD4CEFFE045AEC560A
:104D8000FD0332EC54FD033030C60A3A35DE06E648
:104D9000012709FC0146FE0144BD48F63138DF0613
:104DA00039DE063C3C3C349F06F6032A18DE061822
:104DB000E701FE045AE14E26037E4F5DFE045AF6DB
:104DC00070A418DE0618E703F67001C50227121852
:104DD000E601E14E24035C200D18DE06186A01206E
:104DE00008E64E18DE0618E70118DE0618E6011878
:104DF0006F0418E705CDEE048FC370048FFC70AA12
:104E00003736FC70A8373618EC040505DD02DF04E0
:104E1000DE028FC370248FEC023736EC00DE0437DD
:104E20003618E6033734E600BD4CEFFE045A18305E
:104E3000C60A183A183518DE0618E601E14E2604AF
:104E40005FBD4E32FC0146FE0144BD48F6FE045AE9
:104E500018DE0618E601E14E27037E4EBCBD053B79
:104E600058585858C430DE06E70418CEE66C18E6E9
:104E700000C4CFE702E604EA0218E700FE045AEC99
:104E80004EFD032AEC4CFD032838383138DF063953
:104E9000DE063C3C3C349F06CEE63EE60018DE06CD
:104EA00018E702C504273B18FE045A18E652F1031E
:104EB0002E272FCEE63D58585818DF0418DE061866
:104EC000E703C40818E704E600C4F718EA0418E783
:104ED0000518DE04E70018EC52FD032E18EC50FD17
:104EE000032C38383138DF0639DE063C308FC3FFFB
:104EF000D68F359F06DE083CDE0A3CDE0C3CDE0E1B
:104F00003CDE066F015FE70A6F106F0F6F0E6F0DCB
:104F1000CEE84CCC2000ED024F5FED0018CE000F24
:104F2000183C18CE0000183CCC096FBD4078CC006E
:104F30000F37367F00037F0002DC023736CC0829AA
:104F4000BD4078C6113734CC09FABD403F30C60A9F
:104F50003A35CEE8A3E6002706BD54C67E54AFCE50
:104F6000E8BC18DE06EC0218ED13EC0018ED11CECB
:104F7000E73E1C00041D000418CEE8A8181D00011F
:104F8000CEE888EC02DD0AEC00DD08CEE88CEC020D
:104F9000DD0EEC00DD0CF602D82716CEE89018DF07
:104FA0000418DE06EC0218ED0FEC0018ED0D18DE0B
:104FB00004181C0001CE00013CCE00003CCC096F5F
:104FC000BD4078CC09D4BD40CC84FFC4E08F843F81
:104FD000C4FF8F18DE0618ED08CDEF06CC000F37A2
:104FE000367F00037F0002DC023736CC0829BD4043
:104FF00078CE000F3CCE00003CCC096FBD4078C697
:10500000103734CC09FABD403FCC0137BD40CC1835
:10501000DE0618ED04CDEF0230C60E3A35F602D9A1
:105020007D02D82772D70118DE00188F4F188FDC49
:105030000ADE0818DF02BD5D07DD0ADF08DC0EDED0
:105040000C18DE02BD5D07DD0EDF0CCC00209302E4
:1050500018DE0618ED1518EC0FCE0000183C18EEFF
:1050600015BD5CF418389A0ADA0B8F9A08DA098FA2
:10507000DD0ADF0818CE0010DE02DF00188F930073
:10508000188FDE06EE0D4F5FBD5CF49A0EDA0F8FBF
:105090009A0CDA0D8F2029DE066F25E726DC0ADE62
:1050A0000818DE06183C18EE25BD5D071838DD0A25
:1050B000DF08DC0EDE0C183C18EE25BD5D07183845
:1050C000D30A8FD90999088FDD0EDF0C18DE06CDC3
:1050D000EE083CCDEE063C5FBD56B638385D262264
:1050E00018DE06CDEE133CCDEE113C7F00037F00B1
:1050F00002DD04DC023736DC04DC023736DC047EF9
:1051000053974F0505C301F4188F18EC26CDEE24F4
:1051100018E3228F18E92118A9208FDD0ADF08DCA7
:105120000804DD08DC0A4656DD0A18DE0618EC0421
:10513000CDEE02BD55304F0505C301F4188FDC0ECE
:10514000DE0CD30A8FD90999088F18E3028F18E96A
:105150000118A9008FDD0EDF0CFE0462E60127595D
:10516000EC0A05050505DF00D300C30014DE06EDDB
:1051700017BD5BB518DE0618EE1718ED02CDEF006F
:10518000FE0462EC0A05050505DD0218DE02DF00FB
:10519000188FD300188FDC0E18ED12DC0C18ED10F0
:1051A000EC0A05050505188FDF00188FD300188F4E
:1051B000DE06EC13840318ED18FC0328DE06ED1957
:1051C00004040404ED0BDC0EED29DC0CED2718DFE4
:1051D0000418DE06DC0EDE0C18DF0218DE0418CE22
:1051E0000006BD5D0718DE0218ED29CDEF2718EC8B
:1051F0000BCDEE0BBD5D1A18ED1BDD0018DE0016A1
:105200004F5454188F7F00097F0008183CDC083782
:1052100036DE02EC29EE27BD5C941838183818DF0A
:105220000418DE0618ED1FCDEF1D18E60A18DE047F
:10523000C116224918DE064F18E60A050505C30106
:10524000F48FEC28CDA319260FEC2A1A83006926C7
:1052500007C60118E701200918DE06186F01186C4F
:105260000ADD04DC06DD02DC043CDE026D013826CA
:105270000CDF04DE02E60ADE04C11623B718DE06E0
:10528000186D012629CDEE133CCDEE113C18DE0E33
:10529000183C18DE0C183C4F5FCE0000BD57DBCE2B
:1052A000E204CC2000ED024F5FED007E54A74F18C2
:1052B000E60A050505C302208FEC02DD0CDC0C18A4
:1052C000E31FCDEE1D240108F302D68FF902D5B9F4
:1052D00002D48FDD0ADF08FE0462E60126037E5455
:1052E0006EEC0A05050505DD0218DF0418DE02DF95
:1052F00000188FD300188FDC0A18ED0EDC0818EDAB
:105300000C18DE04EC0A05050505DF00D300C30018
:105310001A8F7D04532704C6032002C601E700FE4E
:105320000462EC0A05050505188FDF00188FD3000D
:10533000188FF676AC18E71BFE046218DE06CDEF78
:1053400021EC0818CEFFFF183CBD37B1DE06EE2178
:10535000ED08FC0462DE06ED23188F18EC0ACDEE92
:1053600006093CBD37B1DE06EE23ED0A3838CEE241
:1053700004CC2000ED024F5FED00FC769EC50127B6
:105380002E18DE0C18DF0E7F000D7F000CDC0A37B4
:1053900036DC08373618DE06CDEE1F3CCDEE1D3C60
:1053A000DC0EDE0CBD3E1C1838183818381838389A
:1053B000DF0E38DF0C38DF0A38DF08308FC3002AF1
:1053C0008F3538DF0639DE063C9F06CEE8A91C0083
:1053D00040CC000F37364F5F3736CC0829BD4078B8
:1053E00018CE000F183C18CE0000183CCC096FBD39
:1053F0004078C6103734CC09FABD403F18CEE8A932
:10540000181D0040CEFFFF3CCE00003CCCFFFF3714
:10541000364F5F3736CCFFFFBD57DBCEE204CC20E2
:1054200000ED024F5FED0030C6123A3538DF063925
:1054300018DE06183C1830188FC3FFE4188F183593
:105440009F0618DE08183C18DE0A183C18DE0C18F7
:105450003C18DE0E183C18DE0618ED1BCDEF198443
:1054600001C400CE0000DD0ADF0818EC1B8402C472
:105470000018ED03CDEF01CDEE194F5F8F8400C40E
:10548000018FDD0EDF0CCDEE198F8400C4028F1862
:10549000ED07CDEF05CDEE198F8400C4048F18ED14
:1054A0000BCDEF09CDEE198F8400C4088F18ED0FD6
:1054B000CDEF0DCDEE198F8400C4208F18ED13CDE4
:1054C000EF11CDEE198F8400C4408F18ED17CDEF8A
:1054D0001518EC1B8400C403CE000026061A8300B6
:1054E00001275A8C000027037E569D1A830003274C
:1054F000037E569DDE082604DC0A2713DE06EE0135
:10550000260818DE0618EC032705C6077E569EDE21
:10551000082604DC0A270CDE0C2604DC0E2704C651
:1055200006207BDE0C2604DC0E2772DE06EE0D263E
:105530000818DE0618EC0F2764C6052061DE082671
:1055400004DC0A2720DE06EE11260818DE0618EC19
:10555000132712DE06EE15260818DE0618EC1727AC
:1055600004C6042039DE082604DC0A2704C603200A
:105570002DDE06EE05260818DE0618EC072712DEDB
:1055800006EE09260818DE0618EC0B2704C60220D2
:105590000DDE0C2604DC0E2704C60120015F4F3807
:1055A000DF0E38DF0C38DF0A38DF08308FC3001C0D
:1055B0008F3538DF0639DE063C3C3C3C9F06DE0872
:1055C0003CDE0A3CDE0C3CDE06E7017F000D6F038B
:1055D000E704EC030505C30214188F18EC02DD0A7A
:1055E00018EC001AA30B25222207DC0A1AA30D25AA
:1055F0001918DE0618EC0DCDEE0B18CE001DBD5DA2
:10560000078C00002604DD0027044F5F2070DE06B3
:10561000EE038C0001276018DE064F18E601DB0D53
:105620008900475618ED0518E7020505C30214184E
:105630008F18EC02DD0A18EC0018DE06CDA30B2251
:105640001E2507DC0ACDA30D241518DE063718E643
:1056500006D70118DE0033188FD70D188F200918D0
:10566000DE0618E60218E701DE064FE601D00D82DD
:10567000001A83000126A018DE064F18E60138DF65
:105680000C38DF0A38DF0838383838DF063918DEDA
:1056900006183C349F0618DE08183C18DE0A183C31
:1056A000DD0ADF08DE066F01DC082607DE0A8C0053
:1056B000012318DE066C01DC0804DE0A8F4656DD85
:1056C0000ADF0826EE1A83000122E8DE064FE60113
:1056D00038DF0A38DF083138DF063918DE06183CB3
:1056E0003C3C3C9F0618DE08183C18DE0A183C18A3
:1056F000DE0C183C18DE0E183CDD0ADF0818DE064A
:1057000018EC0DDD0E18EC0BDD0CFE0462E6012634
:10571000037E58CCEC0A05050505DF00D300C30065
:105720001418ED01BD5BB518DE0618EE0118ED0288
:10573000CDEF00FE0462EC0A05050505DD0218DE6A
:1057400002DF00188FD300188FDC0A18ED0EDC087A
:1057500018ED0CEC0A05050505DD0218DE02DF0078
:10576000188FD300188FDC0E18ED12DC0C18ED101A
:10577000EC0A05050505DF00D300188F186F1AFE27
:10578000046218DE06CDEF03EC08CEFFFF3CBD3708
:10579000B118DE0618EE0318ED08FE046218DE06E6
:1057A000CDEF05EC0AEE06093CBD37B1DE06EE058D
:1057B000ED0AFC04F4C30001FD04F47F00097F003E
:1057C00008CEE844ED02DC08ED003838CC000138A2
:1057D000DF0E38DF0C38DF0A38DF0838383838DFBA
:1057E0000639DE063C9F06DE083CDE0A3CDE0C3C49
:1057F000DE0E3CCC022ABD419EDD0EDF0C4F5F8FDA
:105800008402C4008F18CE0019BD5D07F702D8DCF2
:105810000EDE0C84C0C4008F8400C4038F18CE0039
:105820000EBD5D0758F702D9D60F4F1AB302DA271B
:1058300058FD02DACE0025BD5D1ADD08C6053734F5
:10584000C601BD59CD18DE08183CC601BD5A2CDE74
:10585000083CC608BD5A9918DE08183CC617BD5B3F
:1058600006DE08DF0A7F00097F0008FC02D6FE0280
:10587000D418DE0A183C18DE08183CBD5C94FD0202
:10588000D6FF02D430C60C3A35CEE8A91D0020CE92
:10589000000F3CCE00003CCC0829BD4078CC000F66
:1058A00037364F5F3736CC096FBD4078C610373476
:1058B000CC09FABD403F308FC3000A8F3538DF0E68
:1058C00038DF0C38DF0A38DF0838DF0639DE063CFF
:1058D0003C3C9F06DE06E702E701274718DE064F3D
:1058E00018E6010505C3021018ED03DD02DE02EC27
:1058F00002EE00DD04DC063718E60AD70118DE00E8
:1059000033DD02DC04BD5CF4DF04DE021AEE0318B2
:10591000ED02DE04CDEF00DE026A013CDE02E601AC
:105920003826B9CC0001383838DF0639DE063C3C71
:10593000349F06DE083CDE0A3CDE0C3CDE06EE0848
:10594000DF0C18DE0618E701273DDE064FE60105ED
:1059500005C30214ED027F00097F0008188F18ECC0
:1059600002CDEE0018DE0C183C18DE08183CBD5CB9
:10597000941838183818DE0618EE0218ED02CDEF2C
:1059800000DE066A0126C3CC000138DF0C38DF0ACE
:1059900038DF08383138DF0639DE063C3C349F06F4
:1059A000DE083CDE0A3CDE0C3CDE06EE08DF0C18AE
:1059B000DE0618E701273DDE064FE6010505C301B7
:1059C000F0ED027F00097F0008188F18EC02CDEE81
:1059D0000018DE0C183C18DE08183CBD5C94183822
:1059E000183818DE0618EE0218ED02CDEF00DE06BC
:1059F0006A0126C3CC000138DF0C38DF0A38DF0823
:105A0000383138DF0639DE063C3C349F06DE083C80
:105A1000DE0A3CDE0C3CDE06EE08DF0C18DE061863
:105A2000E701273EDE064FE601050505C30218ED36
:105A3000027F00097F0008188F18EC02CDEE0018D5
:105A4000DE0C183C18DE08183CBD5C941838183879
:105A500018DE0618EE0218ED02CDEF00DE066A0130
:105A600026C2CC000138DF0C38DF0A38DF083831B5
:105A700038DF0639DE063C9F06CEE8A91C0020CCA4
:105A8000000F37364F5F3736CC0829BD407818CE27
:105A9000000F183C18CE0000183CCC096FBD4078B0
:105AA000C6113734CC09FABD403F308FC3000A8F8E
:105AB0003538DF0639DE063C3C3C9F06DE083CDE1E
:105AC0000A3CDE0C3CDE0E3CCEE8B4EC02DD0AEC17
:105AD00000DD0818CEE8B0DF04DE0618EC02ED03A6
:105AE00018EC00ED01DE04EC02DD0EEC00DD0CDE56
:105AF000089C0C2607DC0A1A930E2710DF04DE062A
:105B000018EC02ED0318EC00ED01DE04DC0ADE08FF
:105B100018CE001CBD5CF4DD0EDF0C18DE0618ECA0
:105B200003DD0A18EC01DD08DC0ADE0818CE0004EB
:105B3000BD5D07DD0ADF08DC0EDE0C9A0ADA0B8F8A
:105B40009A08DA098F183818DF0E183818DF0C1881
:105B50003818DF0A183818DF0818381838183818B5
:105B6000DF0639DE063C9F06188F18DF0418DE06B4
:105B7000CDEE0518EC0718DE041A830000270F3657
:105B8000A60018A700081808328F098F26F1188F71
:105B900038DF06393C3736183018EC08272D8C00D2
:105BA0000027398D75CDEE00271B18ED0218EC0685
:105BB00027088D6618E30218ED0218EC088D738F24
:105BC000183018E3028F313131313918EC002707D2
:105BD000CDEE0627038D438F4F5F20EA18EC002798
:105BE000F6CDEE0627078D3218ED0220CD18EC0811
:105BF0008D4020D2188F4FC41F188F2709058F5949
:105C0000498F180926F739188F4FC41F188F270995
:105C10008F048F4656180926F739DF0037D6013D25
:105C20009600D70033373DDB00D7009601333D9B0C
:105C300000393C373630E6063D188FE607323DED39
:105C400002A601E6063DE302E70216183A2406C65C
:105C5000FF183A1808E607323DAB0238183C3824E2
:105C600001083953438F53438F398C00102C0A8C11
:105C700000002704050926FC394F5F390E3E20FC41
:105C80000FCB0CE90D190D320D4B0D640FCB0D022E
:105C90000D920DAB0FC40FC40FC40FC40FC40FC4BB
:105CA0000DC40DDB0DF00DF50DF50DF50E1B0E2FD2
:105CB0000E340E390E3E0FC40FC40FC40FC40FC4F0
:105CC0000E5A0FC40FC40FC40FC40FC40FC40FC4A7
:105CD0000FC40FC40FC40FC40FC40FC40FC40FC42C
:105CE0000FC40FC40FC40FC40FC40FC40FC40FC41C
:105CF0000FC40FC40FC40FC40FC40FC40FC40FC40C
:105D00000E6C0E060E0E0E0E0FC40FC40FC40FC481
:105D10000FC40FC40FC40FC40FC40FC40FC40FC4EB
:105D20000FC40E890E920ED10EE30E9B0EBD0EF522
:105D30000F1F0F330F530F7A0F8C0F9E0FB0472199
:105D40004779472C47794737477947424779471C76
:00000001FF
